:020000040000FA
:06000000E3EF07F012001F
:0600080004EF08F01200F5
:060018000CEF08F01200DD
:0E0020000100E40F0000FE00000002000000DE
:02002E008B92B3
:1000300094920001636B676968696969666B010E78
:100040006A6F1200D9CFE6FFE1CFD9FFE652000177
:1000500063511FE1040108BF1BD0400EE66E600E25
:10006000E66E030EE66E0AEC06F0E552E552E55246
:100070000001010E636FDF6A400EDF5C09E2DF50B2
:10008000EA6AAB0FE96E000EEA22EF6ADF2AF4D7C4
:1000900096D103016051080A01E180D10F0A01E104
:1000A00023D1010A01E118D1030A01E1B4D0010A08
:1000B0006AE0070A5DE0010A01E081D10001020E59
:1000C000AB6F00013A0EAC6F0001010EAD6F000185
:1000D000010EAE6F0001AF6B100EB06FB16BB26B63
:1000E0000001B36B700EB46FB56BB66B0001030EFD
:1000F000B76F0001B86BB96B300EBA6FBB6B000104
:100100000E0EBC6FBD6BBE6BBF6B0001010EC06FEE
:100110000001C16BC26B200EC36FC46B0001080EDF
:10012000C56FC66BC76BC86B0001C9690001020EC1
:10013000C96F0001CA6BCB6BF00ECC6FCD6B0001A9
:10014000CE6B010ECF6FD06BD16B0001D269040171
:100150000CBF0DD0400EE66EAB0EE66E000EE66EE6
:10016000DAEC05F0E552E552E5520001636B27D168
:100170000001010E6A6F0301615102E100016A6B27
:100180000001636B1CD1400E0001646F656B0001C0
:10019000000E645D020E65591FE2040064C000F0A9
:1001A00065C001F0026A060E1F0B00C0F6FF01C019
:1001B000F7FF02C0F8FF06E0D890F636F736F836BB
:1001C000E806FAE1940EA66EA3D964EC06F00001ED
:1001D000642B000E6523DBD7DF6ADF50A96EA868A9
:1001E000040EA66E64EC06F093D9DF50DF2A006E91
:1001F000016A026AFF0E005C000E0158000E0258F0
:10020000ECE3F66AF76A200EF86E940EA66E80D9BB
:100210000001636BD4D0300E0301635D07E1000180
:100220006A5101E132D90001636BC9D0F00E0301BC
:10023000635D04E14DD90001636BC1D0E868000142
:10024000671905E1E868681902E1E868691906E1DB
:1002500061C367F062C368F063C369F0670EE96E5B
:10026000000EEA6EEE500301611908E1EE50030141
:10027000621904E1EE500301631900E12AE1DF6A2B
:1002800003016551DF5C25E23A0E0301D880655514
:10029000DF24EA6A660FE96E030EEA22EF50E66E8B
:1002A00000016651EA6A6B0FE96E000EEA22E55220
:1002B000E750EF6E0001662B0001672B000E6823EC
:1002C000000E6923200E0001665D01E17DD8DF2A62
:1002D000D7D70001636B73D077D80001676968696D
:1002E00069690001636B6BD00001070EAB6F61C3DE
:1002F000ACF062C3ADF063C3AEF064C3AFF065C3EE
:10030000B0F061C3F6FF62C3F7FF63C3F8FFDF6AB3
:1003100003016551DF5C31E2F00E0301635D13E11F
:10032000DF5003016125A96EA66AA6803A0E03017B
:10033000D8806555DF24EA6AB10FE96E000EEA2223
:10034000A8CFEFFF18D00900300EF85C08E1050EC9
:10035000F65C01E1F568080EF65C01E1F5683A0E1D
:100360000301D8806555DF24EA6AB10FE96E000EFB
:10037000EA22F5CFEFFFDF2ACBD704010CBF0DD067
:10038000400EE66EAB0EE66E000EE66EDAEC05F0A1
:10039000E552E552E5520001636B11D06D926D6A32
:1003A000DF6AFF0EDF5C09E2E868E85004E0E80677
:1003B00000D000D0FAD7DF2AF4D7FF0000D0E552F2
:1003C000E552E7CFD9FF12000001EC6B66C000F0E8
:1003D000016A026A00500001675DF66E015000017B
:1003E0006859F76E025000016959F86E1F0EF61435
:1003F0000001ED6FE00EF6160001EB6B200E000120
:10040000EB5D1FE20001ED5115E1000166510FE0C7
:100410000001EC51EA6A6B0FE96E000EEA22EF5020
:10042000F56E0D000001EC2B0001660702D0F568A7
:100430000D0004D0F5680D000001ED070001EB2B65
:10044000DDD70A00A40EA66E63D80001EB6B000195
:1004500066510001EB5D18E20001EC510001EB2553
:10046000EA6A6B0FE96E000EEA22EF50E66E0001B9
:10047000EB51EA6A6B0FE96E000EEA22E552E75093
:10048000EF6E0001EB2BE3D7120061C3F6FF62C3EE
:10049000F7FF63C3F8FF0001EE6B03016551000134
:1004A000EE5D15E23A0E0301D88065550001EE2598
:1004B000EA6A660FE96E030EEA22EF50F56E0C0051
:1004C000C40EA66E25D809000001EE2BE6D7120057
:1004D0000001EF6B030165510001EF5D18E20301BC
:1004E00061510001EF25A96E3A0E0301D8806555D0
:1004F0000001EF25EA6A660FE96E030EEA22EF506B
:10050000A86E040EA66E04D80001EF2BE3D71200EC
:10051000F29E550EA76EAA0EA76EA682A6B2FED7B1
:04052000A69412008B
:0C0524007AD9E6526C5032E1689604016E
:1005300000513C0BE842E8420D0828E1180E021970
:1005400023E1040E031920E1100E026F040E036F65
:10055000DF6ADF50006E016A080E005C000E015871
:1005600013E2DF50EA6A180FE96E040EEA22EF5038
:10057000E66EDF50EA6A100FE96E040EEA22E552D9
:10058000E750EF6EDF2AE5D70ED80AD03FD808D063
:10059000040E6C5C03E1689650D802D0000E01D0C6
:1005A000010EE5523FD139D9E652040104BF046B74
:1005B0000301A86BA06BA16BA66BA76B1EEC04F0EC
:1005C000DF6ADF50006E016A010E005C000E015808
:1005D0001AE20301A15117E1F76ADF34FE0BF73687
:1005E000F66E960EF6260E0EF7220900F5CF00F0F5
:1005F0000800F5CF01F004D001C0FAFF0050F96EF9
:10060000FBDFDF2ADED7B4D8E5520CD1020E03019E
:10061000A05D0EE181D80401180E026F040E036F75
:10062000080E016F00BD02D0C80E05D0880E03D0A1
:10063000D8D8E4D88C0E006F1200040E0001FA5DC9
:1006400009E112C46EFF6E50000802E2050E01D0EF
:10065000030EFA6F0301A00510E111D8020E030189
:10066000A85D03E10401840E06D0040104BD02D09C
:10067000C80E01D0880E046F1200F1EF03F0CDD840
:10068000020EE1260301080EA65D000EA7590DE239
:10069000A6C3DEFFA7C3DDFFA85102E1010E03D010
:1006A000A80506E1020EA86F03D0080EDE6EDD6A13
:1006B000040104930491010EDB500413DFCF05F411
:1006C000000EDB500301A65F010EDB50A75B180E86
:1006D000A46F040EA56F0001FBA30CD097D815E002
:1006E000A2C3F6FFA3C3F7FF0800F5507FD8F6E2D8
:1006F000DB06F4D78BD809E0A2C3E9FFA3C3EAFF66
:10070000EF5074D8F7E2DB06F5D7020EE15C02E2A7
:10071000E16AE552E16E86D080D8020EE126030E32
:1007200004010015E76E010EE7CFDBFF01C4DFFF18
:10073000DE500301A627DD50A723180EA26F040E7A
:10074000A36F64D80EE0A2C3E9FFA3C3EAFFEF5092
:10075000A4C3E9FFA5C3EAFFEF6E68D8F2E2DB06A7
:10076000F0D7020EE15C02E2E16AE552E16E5AD096
:100770006D980301A15105E141D8840E006F040179
:100780001DD0040110AF1CD00301A6510401165D59
:100790000301A7510401175904E216C4A6F317C4B4
:1007A000A7F36DDF0301010EA06F28D8800E006F44
:1007B0000401180E066F040E076FC80E046F1200B6
:1007C0000301020EA06F0401056BC80E046F040143
:1007D000080E016F180E026F040E036FC80E006F33
:1007E00012000301A06B0401046B1200A4C3E9FF13
:1007F000A5C3EAFFEF6E030116EF04F00401080E33
:10080000016F100E026F040E036F1200D9CFE9FFC3
:10081000DACFEAFFEE50ED101200D9CFE6FFE1CFBC
:10082000D9FF1200E552E7CFD9FF1200A42B000E2A
:0C083000A523A22BA323DF06010E12005B
:04083C000401105152
:10084000600BE842E842E842E842E842000901E081
:1008500012001151070A40E00B0A3EE0070A33E09C
:10086000010A23E00B0A1FE0020A1DE0030A19E057
:10087000080A10E0010A0CE00F0A08E0030A01E090
:10088000120012D90001040EFA6F12006DEF04F08D
:10089000A4EF04F009D90301FC0EA26F000EA36FB0
:1008A0000CD0BFEF04F0F1EF04F002D90301A26F06
:1008B000A36BFD0EA227000EA3230001FB930301EF
:1008C000010EA66F1200F4D8EA6AFD0FE96E000E61
:1008D000EA2212C4EFFF12001200800E0401105D24
:1008E00032E11351030A1FE0010A0AE0030A29E179
:1008F000DBD80301D60EA26F0D0EA36F120E1ED011
:10090000B2D88C0EF6260E0EC0D8020E0301F76A7E
:10091000A225F66EA351F7220900F5CFA6F30A002F
:10092000F5CFA7F30ED09FD8900EF6260E0EADD8B9
:10093000A2C3F6FFA3C3F7FF0800F5500301A66F9B
:10094000A76B0001FB831200AFD80F0EE66E710E8D
:10095000E66E0F0EA2D8010EE66EFD0EE66E000EDC
:100960009CD812C4FCF00401125104E10001050EF0
:10097000FA6F12000001060EFA6FC5EF05F00401D0
:10098000186B196B040110511F0B020A0FE0030AC8
:100990000BE0010A18E188D8040118810001FBA1CD
:1009A00012D0040118830FD07FD80DD050D801E0A9
:1009B000010E62D8A4C3E9FFEA6EEF50040B03E016
:1009C0000401010E186F0301A1050AE10301180ECD
:1009D000A26F040EA36F0001FB930301020EA66F2A
:1009E0001200040112050EE110511F0B00090AE16B
:1009F0005BD8030E0401115D03E10001FB8102D00D
:100A00000001FB910401125121E110511F0B02085A
:100A10001DE114510F0B000919E019D801E0010E76
:100A20002BD8030E0401115D02E1840E03D014AF34
:100A300007D0400EA4C3E9FFA5C3EAFFEF6E120082
:100A4000880EA4C3E9FFA5C3EAFFEF6E120030D8F9
:100A50000F0B080DF350016A000F006E040E012207
:100A60001451800B120020D804011251F66EF76A5F
:100A7000D890F636F7361200040DF3500301002427
:100A8000A46F000E0120A56F1200F7220900F5CF18
:100A9000A2F30A00F5CFA3F31200E66ED6EC06F03F
:100AA000E552E552E55212000301010EA16F12005A
:080AB000FBDF040114511200E8
:080AB800040110511F0B01089D
:100AC00001E01200145101E01200060E115D24E154
:100AD0001351230A1FE0010A0DE0030A1BE1DBD8D2
:100AE0000001FC0505E10301FA0EA26F0D0EA36FD4
:100AF000090E0DD0D0D80001FC0505E103016F0EF1
:100B0000A26F0E0EA36F0001FC0504E11D0E030190
:100B1000A66FA76B0001FB8304011051600BE84234
:100B2000E842E842E842E842010801E012001151BF
:100B30000B0A25E0080A17E0090A11E0080A09E093
:100B40000B0A05E0080A01E01200C3EF05F0C4EF4C
:100B500005F0A1D80301A90EA26F030E09D09BD8FE
:100B600013C4A9F3120097D80301AA0EA26F030EB3
:100B7000A36F0001FB930301010EA66F12008BD837
:100B800012C4AAF31200120012000301AB6B1E0E76
:100B9000716E0401400E096F200E0A6F040E0B6F78
:100BA000880E086F0401600E0E6F040E0F6F400E6A
:100BB0000C6F1200D9CFE6FFE1CFD9FFE652FC0E51
:100BC000DB50400805E2400EF36EFC0EF3CFDBFF76
:100BD000DF6AFC0EDB50DF5C0FE2DF5050D8EF50D5
:100BE000E66EDF50EA6A600FE96E040EEA22E55213
:100BF000E750EF6EDF2AEDD7FC0EDBCF0DF4400E91
:100C000004010C170C7D880E0C13E552E552E7CF5A
:100C1000D9FF1200D9CFE6FFE1CFD9FF0301AB6BBB
:100C2000040108BF26D0FC0EDBCF00F00951D880AC
:100C3000005403E2FC0E09C4DBFF0301AB6BFC0EA6
:100C4000DB50AB5D0FE2AB51EA6A200FE96E040E98
:100C5000EA22EF50E66EAB5112D8E552E750EF6E44
:100C6000AB2BEDD70401400E096F0817087D880EE5
:100C700008130301AB51E552E7CFD9FF1200E76E2D
:100C8000FD0EDBCFE9FFFE0EDBCFEAFFE750E926E2
:0E0C9000000EEA2212000301020EA16F1200F4
:020C9E006DA641
:100CA0000CD80001FA0508E16DBA06D0686A696AD5
:100CB00069806988020EFA6F12006D6A696A6D8632
:100CC0000001010EFA6F12000001FA5101E1120059
:100CD00068B425D86DB2120068B038D868B817D893
:100CE00068BA24D8030E0001FA5D01E21200030184
:100CF000AC6B040EAC5D0AE268A608D092EC02F080
:100D0000000901E168960301AC2BF3D71200698456
:100D100068986D82A19AA08A0300A09A12006D9231
:100D2000699468A402D06894FCD7120070A00CD01B
:100D3000800E0401005D07E1840E0401045D03E1FF
:100D400004018C0E006F7090689A12006A6A686ADB
:100D50009F0E6B6E7B0E696E6E6A0F0EE66E710EE5
:100D6000E66E0F0EE66E22D8E552E552E552160EFB
:100D7000706E68A605D0689600D000D00000F9D744
:100D80006D98F1EC03F00401080E016F0401100EE0
:100D9000026F040E036F04018C0E006F0001FB91C3
:100DA0000001FC6B0001030EFA6F1200D9CFE6FFC1
:100DB000E1CFD9FFFD0EDBCFE9FFFE0EDBCFEAFF6F
:100DC000FC0EDB5004E0EE6AFC0EDB06F9D7E552C0
:060DD000E7CFD9FF12007D
:0A0DD6001201000200000008D8041A
:100DE0003C0002000102000109022900010100C0CB
:100DF0003209040000020300000009211101000172
:100E0000221D000705810340000107050103400082
:100E1000010403090434034D006900630072006F8C
:100E200000630068006900700020005400650063E2
:100E30000068006E006F006C006F00670079002092
:100E40000049006E0063002E00260348004900445C
:100E5000002000550053004200200042006F006F48
:100E60000074006C006F0061006400650072000691
:100E700000FF0901A10119012940150026FF007595
:100E80000895408100190129409100C0E80DE80D46
:080E9000110E150E490EB80AFF
:080E9800200EF66E000EF76E4D
:100EA000000EF86E00010900F550F56F0900F550CD
:100EB000F66F03E1F56701D03DD00900F550F06F02
:100EC0000900F550F16F0900F550F26F09000900B3
:100ED000F550E96E0900F550EA6E090009000900B5
:100EE000F550F36F0900F550F46F09000900F6CFD3
:100EF000F7F0F7CFF8F0F8CFF9F0F0C0F6FFF1C057
:100F0000F7FFF2C0F8FF0001F35302E1F45307E0EA
:100F10000900F550EE6EF307F8E2F407F9D7F7C0D1
:100F2000F6FFF8C0F7FFF9C0F8FF0001F507000E63
:060F3000F65BBFD71200C2
:0A0F360082A002D000EF08F00ED8F0
:100F4000040016D819D8060E0001FA5D05E16D50AF
:100F5000020B02E122EC00F0F3D71200140E6F6EC8
:100F60000001FA6B0001FB6B0001FC6B17EF00F056
:100F70004FEC06F064EF06F00001FE51FF1104E1B2
:100F8000100EFE6F270EFF6FFE07000EFF5B060EB2
:100F90000001FA5D02E28B8212000001FE51FF1196
:060FA00001E18B7212005A
:0A0FA600000EF36E00EE00F0080EDE
:100FB00001D81200EA6002D0EE6AFCD7F350E96073
:060FC0001200EE6AFCD7EE
:0A0FC60013EE00F023EE00F0F86ACD
:100FD000049C4CEC07F0F1EC07F09BEC07F0FBD71E
:020FE0001200FD
:020FE2001200FB
:020FE40000000B
:020000040030CA
:01000000E41B
:010001003EC0
:01000200F904
:01000300FEFE
:01000500F901
:010006009B5E
:01000800FFF8
:01000900FFF7
:01000A00FFF6
:01000B00FFF5
:01000C00FFF4
:01000D00FFF3
:00000001FF
